:020000040000FA
:020000005D2879
:08000800FE00030EFD000408D8
:10001000FF000A08FC008A01830183011A08E0003E
:100020006430E100850A85110610E01D06146008A1
:10003000FF3C03195228411D482841116008FE3C2D
:10004000031946286008F13C031933286008F03C86
:1000500003193F286008F63C031939286008F83C6A
:100060000319392853280130C7000830C800C116C9
:1000700053280030C7000130C800C1165328033090
:10008000E1000830E000BE23C1125328FF30E00039
:100090004808003C03193F28BE23C70A031D532804
:1000A000C80A532841158C127F0884007C088A00F6
:1000B0007D0E8300FE0E7E0E09008316031383302F
:1000C0008100F0308500323086009F018E01CF30F4
:1000D000990020308C0022309800830107309F0067
:1000E0001A08E0001A08E000903098008C01C03037
:1000F0008B00C116C7010830C8002030E000BE23C5
:10010000CF23C11264009F24C7010830C800E10159
:10011000CC0141160430C900C1116108003C03192B
:100120009C286108013C03198228E103FA30C200CF
:100130008611EB2386158D28F82383173F30840022
:10014000861164000614801F061084038615841A25
:10015000A0288301BF308400861164000614801F2C
:10016000061084038615841AAC283F30840086115B
:1001700064000614801F061084038615841AB728AD
:1001800083010330C200EB2306308500DE23F82311
:1001900083173F308400861164000614001F061088
:1001A00084038615841ACB288301BF30840086110E
:1001B00064000614001F061084038615841AD728CD
:1001C0003F308400861164000614001F061084036B
:1001D0008615841AE22883010330C200EB2307301E
:1001E0008500DE23F82383173F30840086116400E6
:1001F0000614801E061084038615841AF6288301CF
:10020000BF308400861164000614801E061084032B
:100210008615841A02293F30840086116400061472
:10022000801E061084038615841A0D29830103306D
:10023000C200EB2302308500DE23F82383173F3012
:100240008400861164000614001E061084038615BF
:10025000841A21298301BF308400861164000614AA
:10026000001E061084038615841A2D293F30840051
:10027000861164000614001E061084038615841A75
:10028000382983010330C200EB2303308500DE23CD
:10029000F82383173F308400861164000614801D04
:1002A000061084038615841A4C298301BF3084000C
:1002B000861164000614801D061084038615841AB6
:1002C00058293F308400861164000614801D0610F2
:1002D00084038615841A632983010330C200EB234B
:1002E00005308500DE23F82383173F308400861114
:1002F00064000614001D061084038615841A7729ED
:100300008301BF308400861164000614001D0610AE
:1003100084038615841A83293F3084008611640083
:100320000614001D061084038615841A8E29830185
:100330000330C200EB2300308500DE23F82383174F
:100340003F308400861164000614801C061084036C
:100350008615841AA2298301BF30840086116400A7
:100360000614801C061084038615841AAE293F30BB
:100370008400861164000614801C06108403861510
:10038000841AB92983010330C200EB2304308500AD
:10039000DE23F82383173F3084008611640006149F
:1003A000001C061084038615841ACD298301BF30F2
:1003B0008400861164000614001C06108403861550
:1003C000841AD9293F308400861164000614001C69
:1003D000061084038615841AE42983010330C200C1
:1003E000EB2301308500DE234D08003C031D532A1A
:1003F000CB2479082F3C031D2C2AF701E401BF24EC
:10040000CB247908CD00BF22BF24CB243030F902A1
:100410000730F9054D08733C0319222A4D08533C57
:100420000319222A790ECE00F030CE053230CE07E5
:100430002030F900292A41127909C9000730C9057D
:10044000CD01292A41167909C9000730C905CD0116
:10045000292ABF24CB24CC017908083C031D352A66
:10046000C7010830C8002030F900DE247908DB3CE1
:1004700003194A2A7908FB3C03194A2A7908203CC7
:1004800003194A2A4C08023C03184A2A7808003CFF
:1004900003194F2ACC0A4C08083C031D512ACC01F1
:1004A000BF24C119F809411A612AC30A4908F60094
:1004B000F60D76101530F60743087602031D8D28D9
:1004C000C3014D08443C03198C2A4D08643C0319B0
:1004D0008C2A4D08553C03199A2A4D08753C03197E
:1004E0009A2A4D084A3C0319A82A4D086A3C031968
:1004F000A82A4D08573C0319B02A4D08773C031928
:10050000B02A4D08463C0319B52A4D08663C03192C
:10051000B52ACD0147248D28F70A7708033C031D2F
:100520008D28F7012623E40A64080A3C031D8D2860
:10053000CD018D28F70A7708033C031D8D28F701AC
:10054000FA22E40A64080A3C031D8D28CD018D2897
:10055000FD23E40A6408323C031D8D28CD018D285B
:10056000CE03031D8D28CD018D28FF30F8004724D0
:10057000E40A6408603C031D8D28CD018D284D08D8
:10058000493C0319F02A4D08693C0319F02A4D082B
:100590004E3C0319F32A4D086E3C0319F32A4D080B
:1005A000513C0319F62A4D08713C0319F62A4D08EF
:1005B000443C031908004D08553C031908004D0838
:1005C0004A3C031908004D08573C031908004D0820
:1005D000463C031908004D08533C03190800080065
:1005E000C115CD010800C111CD0108007D2457308F
:1005F000CD000800CF0120308400841383134F08FE
:100600008407800C8013CF0A4F08203C031DFB2A6F
:10061000CF0120308400841783134F088407800C97
:100620008013CF0A4F08203C031D092BCF01203037
:100630008400841383174F088407800C8013CF0A2B
:100640004F08203C031D172B83010800CF012030E9
:100650008400841383134F088407800D0010CF0A91
:100660004F08203C031D272BCF0120308400841726
:1006700083134F088407800D0010CF0A4F08203CD9
:10068000031D352BCF0120308400841383174F08BE
:100690008407800D0010CF0A4F08203C031D432B18
:1006A000830108008617831603138613831203132E
:1006B00006130000000000000617000000006400A0
:1006C0000000000086130000000000000000000091
:1006D00006130000000000348613831603138613EC
:1006E00083120313861300000000000006170000A9
:1006F00064000000861700000000000006130000E0
:1007000000000000061700348316031386138312BB
:100710000313721F8D2B86178F2B8613000006176D
:10072000000000006400000006130034F217831676
:1007300003138617831203130617000000006400DA
:1007400000000000861FF213061300340830F50085
:100750007213F41B72178423F40DF50BA82B962348
:100760000034F0010830F5000310F00D9623F21B61
:100770007014F50BB52B721784230034C11E0800CA
:100780005223A030F400A6234808F400A62347080B
:10079000F400A6236008F400A6236C23080032307E
:1007A000E2006E30E3000000000000006400000082
:1007B0000000E30BD32BE20BD12B0034411EE82BBE
:1007C0004908F6000530F607E823F60BE42B08008D
:1007D000FF30C200EB2B6400C20BEB2B0800613032
:1007E000F6000610861164008615F60BF22B080041
:1007F000830185153730C200EB2B83012030840044
:1008000084138313840A000884038000840A040884
:100810003F3C031D022C8301831620088301BF0087
:10082000A0308400840A000884038000840A04083D
:10083000AF3C031D122C831603137808AF0083010D
:100840003F3084008413831784030008840A8000E7
:1008500084030408203C031D242C831603133F0843
:1008600083120317A00083013F3084008417831391
:1008700084030008840A800084030408B03C031D3C
:10088000382C831603137808B00083010800830115
:1008900020308400840A000884038000840A04084D
:1008A0003F3C031D4A2C8301831620088301BF00AF
:1008B000A0308400840A000884038000840A0408AD
:1008C000DF3C031D5A2C83010317200883160313F2
:1008D000BF0083012030840084138317840A00083A
:1008E00084038000840A04083F3C031D6E2C83129D
:1008F00003177808BF0083010800640020308400DB
:10090000841383138001840A0408403C031D822C55
:1009100020308400841783138001840A0408C03CBB
:10092000031D8C2C20308400841383178001840ADB
:100930000408403C031D962C64008301080020300D
:100940008400841383138001840A04087F3C031D00
:10095000A32C20308400841783138001840A0408A8
:10096000FF3C031DAD2C20308400841383178001CD
:10097000840A04087F3C031DB72C83010800C70AC2
:10098000031D0800C80A4808003C031D0800C701F1
:100990000830C80008005223A030F400A6234808FD
:1009A000F400A6234708F400A6235223A130F40044
:1009B000A623B1236C237008F90008007908F5001C
:1009C000F50DF50D750DCA00F830CA054C08CA07BB
:1009D000F90E790C0739CB005223A030F400A6237E
:1009E0004B08F400A6234A08F400A6235223A130A2
:0E09F000F400A623B1236C237008F800080061
:020FFE000000F1
:02400E000603A7
:00000001FF
